:020000000628D0
:080008000B11090005308C000A
:1000100009308D000A308E0006308F0000309000CD
:1000200083160030860083120130003C03193F28FC
:1000300000309A000C301A02013003180001003C15
:10004000031928283230990073207C209A0A1A2834
:1000500003309700582000309A000C301A0201300B
:1000600003180001003C03193B2889203230990015
:1000700073209A0A2D28033097005820142811085D
:1000800092001430930000000000930B4328920B61
:100090004128140896006E30950000000000000012
:1000A000000000000000950B4D28960B4B2808001F
:1000B0001708003C013003190001003C03197228A5
:1000C000003098000A301802013003180001003C8B
:1000D00003196F28643094004920980A6228170891
:1000E00097035828080010080C3E8400000886007A
:1000F00019089400492008001008900A1008043CD0
:100100000130031D0001003C0319882800309000D5
:1001100008001008003C0130031D0001003C0319D9
:0E0120009428033090009628100890030800E1
:00000001FF
